:100000008316033085008601831291019F01B72872
:1000100082073F3430345B344F3466346D347D3482
:1000200007347F346F346E343F343E340034383418
:100030003F346D3479340034FF340C088F000230C3
:100040000F06031D262801309000080003300F061C
:10005000031D2D2802309000080004300F06031DF8
:10006000342803309000080005300F06031D3B289C
:100070001108900008008F038F038F038F031F2840
:100080008D018E010C088F008F0A8F0B4828080005
:100090008D0A0A300D06031D45288E0A8D0145285C
:1000A00060309B00000000009A0B522805185C2865
:1000B0001F109B0B522808001F1859288C0304306E
:1000C00093009F141F14592800300E060319772837
:1000D0000E08082086005020860150200D080820B8
:1000E00086005020860150205020502008000D0826
:1000F000082086007328403086009720972006301D
:10010000860097209720972097200D309200860137
:100110009720120808208600FF3006060319B7282A
:10012000920A9720972087280A309200872800009B
:100130009A0B97289B0B9728080001301006031D87
:10014000A42880308600AD2802301006031DAB289D
:10015000C0308600AD28E03086000A309C000000E8
:100160009A0BAF289B0BAF289C0BAF2808001630CA
:100170008C00910A043011060319DD284020642008
:100180009F1CB928930BB9281D209D204020642076
:1001900000300C0603197B288C03900BC6289F1097
:1001A00000300C0603197B2801300C060319942833
:1001B00002300C0603197B28B9289101910ABE2848
:00000001FF
